:020000040000FA
:1000000001288316FF23900008308500003081000E
:1000100008309600831285010730990008308B0064
:100020000630A8009020782085016E209020512075
:100030006E2085016E20902051206E2085016E205B
:1000400090205120851D222874201E30A500643088
:10005000A6009B30A7000C30A400851D3F28A40BF0
:100060002D28A70B2B28A60B2928A50B27285120C4
:100070007120512085010B1063000000122806300A
:10008000A4072408A9007F20682085194828432850
:100090007F207420851D4128A90B48287B209320B0
:1000A00022283030A00085165A2085125A20A00B35
:1000B000532808003030A100A10B5C28080008304C
:1000C000A2007D30A300A30B6328A20B61280800C7
:1000D0005F205F205F205F205F200800682068208D
:1000E00008006E206E2008006E207120712008002C
:1000F00074207420080078207820782008002808D0
:10010000882085005120A80B08000630A8000800B0
:1001100082071F340F341D340D341C340C34183452
:100120001730850008005120712051207120512086
:0A01300071205120712051200800B9
:0207FE0038348D
:02400E00843FED
:00000001FF
